:1000000012C02BC02AC029C028C027C026C025C0C6
:1000100024C023C022C021C020C01FC01EC01DC0DC
:100020001CC01BC01AC011241FBECFE5D4E0DEBF28
:10003000CDBF10E0A0E6B0E0EAE8F4E002C0059031
:100040000D92A036B107D9F710E0A0E6B0E001C0EC
:100050001D92A036B107E1F77BC0D2CF40E050E05F
:100060004817590768F420E030E0275E3F4F60E70B
:100070002E343607D0F34F5F5F4F4817590798F378
:10008000089580B7846080BF87B38F6387BB88B3D0
:10009000817E816288BB84B3837C836084BB85B3AB
:1000A000807C85BB81B384EF81BB82B380E282BB5D
:1000B000089586B186E886B987B184E487B9089542
:1000C0000F931F93369A3699FECF24B185B19927A5
:1000D000182F0027020F111DC801AA2797FDA09510
:1000E000BA2FBC01CD0137D117FF05C020E030E0A9
:1000F00040E857E483D09B01AC0160E070E080E809
:1001000094E4C6D0DC01CB0120E030E040E85FE3BE
:10011000BC01CD0172D0DC01CB0120E030E04CE726
:1001200052E4BC01CD0163D1DC01CB0120E030E021
:1001300040E05FE3BC01CD0161D0DC01CB01BC013B
:10014000CD01ECD0DC01CB0199271F910F910895CF
:10015000CFE5D4E0DEBFCDBF85B5887F85BD91DF1B
:10016000A8DF8B9A939A96989298C09800E010E036
:10017000A7DF992784309105E9F08530910534F4A3
:1001800081309105E1F00297B9F01BC080319105F3
:1001900059F0813191051CF4089749F012C08097FD
:1001A00081F401E010E00DC002E010E00AC003E0BD
:1001B00010E007C08C0105C005E010E002C006E0B9
:1001C00010E00115110559F0E801929A88EC90E0D1
:1001D00045DF929888EC90E041DF2197B1F7012B41
:1001E00041F4C09A88EC90E039DFC09888EC90E048
:1001F00035DF88E592E032DFB9CF5058192ED5D0DF
:1002000001D0B8C0BA176207730784079507B1F128
:1002100088F40EF410940B2EBA2FA02D062E622F08
:10022000202D072E732F302D082E842F402D092EC0
:10023000952F502DFF275523B9F0591B49F0573EF4
:1002400098F0469537952795A795F0405395C9F7AF
:1002500076F0BA0F621F731F841F30F4879577956D
:100260006795B795F040939517FA0F2E0895BF1B29
:10027000BB27BA0B620B730B840BF6CFDEF6B1C053
:10028000592F482F372F262F9FE380E8772766279F
:100290008CD001D06FC0552359F0992369F09F5736
:1002A0005F57951B33F442F4903811F4915805C010
:1002B00079C091589F3F09F494C0BB27112462175D
:1002C0007307840730F4660F771F881FBB1F915098
:1002D00098F311D00F920FD00F920DD0A0E82617EF
:1002E000370748071B0609F0A048BA2F602D7F91F9
:1002F0008F9100240895A0E80024621773078407F3
:10030000B10528F0621B730B840BB1090A2A660F32
:10031000771F881FBB1FA69581F7089597FB51D0C3
:100320009F3738F0FEE9F91B982F872F762F6B2F18
:1003300005C054C09695879577956795F150D0F78D
:100340003EF490958095709561957F4F8F4F9F4FAC
:100350000895E89403C097FB0EF4F3DFB62F672FE0
:10036000782F892F9EE9002405C09A95BB0F661F40
:10037000771F881F11249923A1F08823B2F79F3F8C
:1003800059F0BB0F48F421F4002011F460FF04C0C1
:100390006F5F7F4F8F4F9F4F881F9795879597F976
:1003A00008951CC09FEF80EC0895052E092607FADA
:1003B000440F551F5F3F79F0AA27A51708F051E0B9
:1003C0004795880F991F9F3F31F0BB27B91708F059
:1003D00091E0879508959F919F91E4CF66277727B5
:1003E000882799270895592F482F372F262FDDDF8B
:1003F00001D0C0CF992339F0552329F09F575F577B
:10040000950F13F4CAF1EDCF91589F3FE1F3A62F5A
:1004100000241124BB2766275527F8E0A69520F471
:10042000020E131EB41F651F220F331F441F551FDA
:10043000FA95A1F7F8E0E72F7727F8E0E69520F4A2
:10044000130EB41F651F7A1F330F441F551FAA1FB9
:10045000FA95A1F7F82F8827F69520F4B40F651FB9
:100460007A1F8E1F440F551FAA1FEE1FFF23A1F7EF
:1004700088231AF4939539F495CF000C111CBB1FF7
:0A048000661F771F881F01280895EA
:00000001FF
